:100000000C94E8000C9468050C9405010C9405010F
:100010000C9405010C9405010C9405010C94050148
:100020000C9405010C9405010C9405010C94050138
:100030000C9405010C9405010C9405010C94050128
:100040000C9405010C9405010C9405010C94050118
:100050000C9405010C9405010C9405010C94050108
:100060000C9405010C9405010C9405010C940501F8
:100070000C9405010C9405010C9405011102130266
:10008000160218021B021D0220022202250227026C
:1000900029022C022E0230023202340236023802C9
:1000A0003A02AD02AD02AD02AD023C023E02400298
:1000B0004202AD02AD02AD02AD0244024602480268
:1000C0004A024C024E025002520254025602580298
:1000D0005A025C025E0260026202AD02AD02AD0233
:1000E000AD0264026602AB0268026A026E0271022D
:1000F000750278027E027B0277027A027D0280021C
:1001000082028402860288028A028C028E02900297
:1001100092029402960298029A029C029E02A00207
:10012000A202AD02AD02AD02AD02A702A402A60278
:10013000AA02BA02BE02BC02C002C602CD02CF02AF
:10014000D102D302DD02E0023403360338033A035E
:100150003C033E03400342034403460348034C036D
:10016000090212000101008096090400000000004D
:10017000000012011001FF000008C016DC0500029B
:10018000010200011E0349004E004C0020005200F5
:100190006500740072006F002D00500072006F0047
:1001A00067002A0349006E00660069006E0069005E
:1001B000740065004E00650073004C006900760015
:1001C000650073002E0063006F006D0004030904D6
:1001D00011241FBECFEFD4E0DEBFCDBF11E0A0E001
:1001E000B1E0EAE4FDE002C005900D92A230B10753
:1001F000D9F711E0A2E0B1E001C01D92A533B1072B
:10020000E1F70E947C060C94A3060C94000011B840
:100210008FEF82B914B885B917B888B98AB18471DB
:100220008AB98BB18B6E8BB9509858985198599A5E
:1002300008950E940701399A419A389A40983A9A4B
:10024000429A3C9A449A3D9A459A3F9A479A4798CF
:100250008FEF84B915B8479A479814B812B881B986
:1002600014B885B95998519A08950E940701399A8E
:10027000419A3C9A449A3D9A459A509A589A3F9A84
:10028000479A4798579A5F9A5F988FEF84B915B845
:10029000479A479814B884B915B85F9A5F9814B80C
:1002A00012B881B914B885B95998519A0895813016
:1002B00049F028F0823051F40E94350105C00E94B7
:1002C000070102C00E94190180E0089586E908959F
:1002D0009FEF94B985B9479A479862B945B958983C
:1002E000509A5098589A14B8089550985898409831
:1002F000419A429A62B99FEF94B985B9479A479853
:1003000014B800000000409A87FD419800000000EA
:10031000000000000000000083B14098419A089559
:1003200062B99FEF94B985B9479A479814B8409A33
:1003300087FD4198000000000000000083B1409854
:10034000419A08955898509A9FEF94B962B985B927
:10035000479A4798429845B9409A87FD41980000CE
:1003600000004098419A429A14B8089562B98032C8
:1003700020F48FEF84B915B803C09FEF94B985B905
:10038000479A479814B84498000000000000000005
:1003900083B1449A0895CF93DF93982F862F642FCB
:1003A000E901913839F0923851F0903859F40E94AF
:1003B000750102C00E949001888380E004C00E9401
:1003C000B601FACF81EADF91CF9108959FEF94B9FA
:1003D00062B9803210F415B801C085B9479A4798C0
:1003E00045B945980000459A14B80895982F862F6E
:1003F000642F422F992329F0913039F40E94E601AD
:1004000002C00E94680180E0089580EA089590E0AB
:100410008B35910508F0A1C0FC01E25CFF4F0C9404
:100420009D0611B895C08FEF81B992C012B890C0E7
:100430008FEF82B98DC014B88BC08FEF84B988C09C
:1004400015B886C08FEF85B983C017B881C018B8BA
:100450007FC08FEF88B97CC038987AC0389A78C04E
:10046000409876C0409A74C0399872C0399A70C06A
:1004700041986EC0419A6CC03A986AC03A9A68C076
:10048000429866C0429A64C03B9862C03B9A60C082
:1004900043985EC0439A5CC03C985AC03C9A58C08E
:1004A000449856C0449A54C03D9852C03D9A50C09A
:1004B00045984EC0459A4CC03E984AC03E9A48C0A6
:1004C000469846C0469A44C03F9842C03F9A40C0B2
:1004D000479A3EC08AB184718AB93AC08BB184719F
:1004E00002C08BB18B6E8BB933C0509831C0589815
:1004F000509A2EC05098589A2BC05098589828C09F
:10050000519826C0519A24C0599822C0599A20C0A7
:1005100053981EC0539A1CC05B981AC05B9A18C0AF
:10052000559816C0559A14C05D9812C05D9A10C0B7
:1005300056980EC0569A0CC05E980AC05E9A08C0C3
:10054000579806C0579A04C05F9A02C05F9A5F9896
:1005500080E00895479A4798FBCF8CE8089590E093
:10056000FC01E058F109EB30F105A0F5E756FF4F2B
:100570000C949D0662B922C08FEF84B965B91EC084
:100580008FEF84B965B9479A479805C08FEF84B952
:1005900065B95F9A5F9814B811C061B90FC064B9AA
:1005A0000DC067B90BC09AB1862F846189238AB9BF
:1005B0008AB16B7E682B6AB901C068B980E0089582
:1005C0009BB1862F846189238BB98BB16B7E682B9D
:1005D0006BB9F4CF8DE80895813A61F0823AB9F0B1
:1005E000803A11F58FEF84B965B9479A479814B8E6
:1005F00042B916C08FEF84B965B9479A479814B8C5
:1006000042B967FF02C041980BC0419A09C042B984
:100610008FEF84B9603230F415B8479A479814B810
:1006200080E0089565B9F9CF8EE80895803B61F4C4
:1006300022B98FEF84B945B9479A479865B95F9A4F
:100640005F9814B880E008958FE80895CF93DF9302
:10065000EB0190E0805C91098C309105F8F48C55A9
:100660009F4FFC010C949D0680B113C083B111C053
:1006700086B10FC089B10DC082B10BC085B109C070
:1006800088B107C08BB105C081B103C084B101C07E
:1006900087B1888380E003C08AB1FBCF80E9DF9116
:1006A000CF9108950F93811102C0589A01C05898B4
:1006B0008FEF84B922B945B9479A479805B96111B6
:1006C00001C04198459800000000459A419A14B82D
:1006D00058980F9108950F93022F813061F030F0F8
:1006E000823089F4242F462F6FEF08C0242F462F25
:1006F00060E081E004C0242F462F60E080E00E948B
:10070000520380E001C08AEA0F9108950F9381118E
:1007100002C0589A01C058988FEF84B902B925B920
:10072000479A479845B95F9A5F9814B8611101C01C
:1007300041984498000000000000000083B1449AF2
:10074000419A58980F9108950F931F93CF93DF9379
:10075000E801813851F0823891F08038A9F4022FF5
:10076000242F462F60E081E005C0022F242F462F62
:1007700060E080E00E948603888380E006C0022F4C
:10078000242F462F6FEFF5CF8BEADF91CF911F918A
:100790000F9108950F931F93CF93FC01C081CC1F3D
:1007A000CC27CC1F8181823049F118F4813031F09F
:1007B00056C0833039F18430A9F151C08281803B29
:1007C00038F4803A88F4803858F40E94070248C010
:1007D000803C78F42481458163810E94160340C0E7
:1007E00064810E94AF023CC0448165810E94EC029A
:1007F00037C063E071E00E9426032DC082810E9411
:1008000057012EC08281803830F423814481658174
:100810000E94F60125C023E031E0448165810E94F9
:10082000CB0119C02281638144817581822F90E0C0
:10083000203840F4262F30E050E0672F70E00E940F
:100840006B030EC0242F30E0472F50E070E003E030
:1008500011E00E94A40380930201CF5F03C080E8EF
:100860008093020182E091E090931A018093190134
:100870008C2FCF911F910F91089581E00895CF9310
:10088000DF9360911B01635067FDA4C08091180144
:10089000CCE0D0E0C81BD109C15EDE4F80911701CA
:1008A0008D3209F085C0683009F092C083EC8093E6
:1008B0000B018AE58093010110920A0188818076FC
:1008C00021F0CE010E94CA0360C08A8110921401F7
:1008D0009981911106C01092150124E131E082E066
:1008E00050C0953019F480931C013DC09630A9F595
:1008F0009B81913019F482E791E004C0923041F479
:1009000080E691E090931A018093190182E121C061
:100910009330F1F4811108C08CEC91E090931A01AE
:100920008093190184E015C0813041F482EA91E09E
:1009300090931A01809319018AE20BC0823041F42E
:1009400084E891E090931A01809319018EE101C02F
:1009500080E090E490930A0118C0983079F09930C3
:1009600031F480931E0124E131E080E00AC081E08F
:100970009A3009F080E024E131E003C02EE131E05B
:1009800081E030931A01209319018F3F39F4988147
:1009900097FD8E8190E890930A0107C09F81911185
:1009A00004C09E81981708F4892F8093000110C01D
:1009B00080910A0187FF0CC0CE010E943D048F3F49
:1009C00021F48EE18093010103C081111092000196
:1009D00010921B018091010184FF4DC080910001A4
:1009E0008F3F09F448C0C82F893008F0C8E08C1B3D
:1009F0008093000180910B0198E8892780930B0177
:100A0000CC2361F18091190190911A0120910A0182
:100A100026FF12C0ACE0B1E02BE031E0209530952C
:100A2000280F391F4C2F4A0FF901EA0FFB1FE491E1
:100A3000ED934A13F9CF09C0ECE0F1E0DC012C2F73
:100A40002E0F3D9131932E13FCCF01962FEF2C0FDB
:100A5000820F911D90931A01809319016C2F8CE0E5
:100A600091E00E946405CC5FCC3019F08FEF809349
:100A70000001C093010184E199B1947131F4815076
:100A8000D9F710921C0110921601DF91CF910895B1
:100A9000E9E6F0E0808182608083E89A0895A82FDB
:100AA000B92F80E090E041E050EA609530E009C065
:100AB0002D9182279795879510F084279527305E92
:100AC000C8F36F5FA8F30895EADF8D939D930895AF
:100AD000CF93CFB7CF93DF93C3954C9BE9F74C9B54
:100AE0000BC04C9B09C04C9B07C04C9B05C04C9B4A
:100AF00003C04C9B01C089C06F93C0911801DD27D2
:100B0000C15EDE4F2F9365E54C9B03C02F916F9123
:100B1000E6CF0F931F934F9320E040E15F9309B11D
:100B2000047104FB27F93F9350E03BE039C0147196
:100B300040642F77012F5F5F1EC0406819B11471A8
:100B40002F7752501FC0406409B12F770471D1F143
:100B50005F5F00C023C0406219B12F77147191F11B
:100B60005F5F00C025C004711027515012F45D5F13
:100B70000000115027952C3F19B1C8F614710127B8
:100B8000015027952C3FC8F64227499309B10471BB
:100B900010274F73115027952C3FA8F64695469580
:100BA00019B1147179F00127015027952C3F98F65F
:100BB0006B5A60F3315009B1B0F600C011E01CBBB4
:100BC000002717C03B503195C31BD04011E01CBB20
:100BD0000881033CF9F00B34E9F0209116011981EA
:100BE000110F1213EDCF093651F10D3211F0013E04
:100BF00039F700931D013F915F914F911F910F9124
:100C00002F916F91CCB3C0FD67CFDF91CF91CFBF54
:100C1000CF91189520911D01222369F310911B019A
:100C2000112339F534303AF130931B012093170129
:100C3000109118013BE0311B309318011CC000914A
:100C40001B010130B4F40AE53091010134FD14C0F8
:100C500000930101CBE0D1E013C0052710E000C0F4
:100C600000000BB91AC0052710E0221F1DC010E0BC
:100C700021C04AE502C032ED432FC4E1D0E032E0AA
:100C80001AB114615C9A0BB11AB954E120E865E31A
:100C900020FF05270BB9279517951C3FF0F66695A1
:100CA000B8F7B1F720FF05270BB9279517951C3F1B
:100CB000D0F62795179517FF052700001C3F0BB9A5
:100CC000B0F629913A9519F70B7E10911C01110F7E
:100CD000C651D0400BB911F01093160111E01CBBA6
:100CE00000611AB11B7E402F4B7E54E05A95F1F7FC
:100CF0000BB91AB94BB97FCF2EE088E190E00FB65F
:100D0000F894A895809360000FBE209360000E9425
:100D10004805549A80E0815041F0A895EFE9FFE042
:100D20003197F1F700C00000F6CF54980E940701F8
:100D30007894A8950E943F04FCCFEE0FFF1F05900A
:0A0D4000F491E02D0994F894FFCF20
:020D4A00FF5A4E
:00000001FF
